:020000040000FA
:100000002F090E0C02002F09000C2500000C260001
:10001000FF0C0500F30C06007F0C32007F0C330050
:100020000605980AAC0C2C0012022D006605000093
:100030000000ED02170A00000000EC021B0A660433
:10004000AC0C2C0013022D00460500000000ED0250
:10005000250A00000000EC02290A46040008FA0CF8
:100060002C000000EC02310A0008000C2E00AC0C41
:100070002C004506390A45073B0A00000000EC0247
:100080003D0A4507470AEE03410AFF0C2E001209FC
:10009000000C2F00AC0C2C0065064C0A65074E0ABC
:1000A00000000000EC02500A65075A0AEF03540AE8
:1000B000FF0C2F00120900080C022D007F0CAC0071
:1000C0004306760A0306710A7F0C2C000D02AC0071
:1000D00003042C030C022D007F0C2C000D02AC003D
:1000E000000803042C037F0CEC0100080D022C0017
:1000F00000080C022D007F0CAC004306950A030695
:100100008C0A7F0C2C000D02AC0003042C030304AA
:100110002C030D02EC01000803042C0303042C0340
:100120000C02AD000D022C0000080D022C0000088E
:10013000350904000604C607AC0AE607A60A0E0243
:100140002C005C095C090C022E00B30A0E022C0084
:1001500079090C022E00B30AE607B30A0E022C003E
:100160005C090C022E002607C40A0507BE0A0F020E
:100170002C005C095C090C022F00CB0A0F022C003A
:1001800079090C022F00CB0A0507CB0A0F022C00BD
:100190005C090C022F000E0230000F0231007F0CB0
:1001A000B0007F0CB100110232001002F2010E0209
:1001B0002C000F02EC010307E30A7F0CAC000307DD
:1001C000E30A800C32000E022C000F02EC01030641
:1001D000EF0A7F0CAC000306EF0A820C320011021A
:1001E00033001002B3000E022C000F02AC00030714
:1001F000FF0A7F0CAC000307FF0A820C33000F02DA
:100200002C000E02AC0003070B0B7F0CAC000307A5
:100210000B0B800C33007F0CF2014306B2027F0C03
:10022000F3014306B30286071D0BFF0C2C001202DC
:10023000AC000C0232004306B202A607980AFF0C7B
:100240002C001302AC000C0233004306B302980AE0
:10025000FF0FFF0FFF0FFF0FFF0FFF0FFF0FFF0F2E
:10026000FF0FFF0FFF0FFF0FFF0FFF0FFF0FFF0F1E
:10027000FF0FFF0FFF0FFF0FFF0FFF0FFF0FFF0F0E
:10028000FF0FFF0FFF0FFF0FFF0FFF0FFF0FFF0FFE
:10029000FF0FFF0FFF0FFF0FFF0FFF0FFF0FFF0FEE
:1002A000FF0FFF0FFF0FFF0FFF0FFF0FFF0FFF0FDE
:1002B000FF0FFF0FFF0FFF0FFF0FFF0FFF0FFF0FCE
:1002C000FF0FFF0FFF0FFF0FFF0FFF0FFF0FFF0FBE
:1002D000FF0FFF0FFF0FFF0FFF0FFF0FFF0FFF0FAE
:1002E000FF0FFF0FFF0FFF0FFF0FFF0FFF0FFF0F9E
:1002F000FF0FFF0FFF0FFF0FFF0FFF0FFF0FFF0F8E
:10030000FF0FFF0FFF0FFF0FFF0FFF0FFF0FFF0F7D
:10031000FF0FFF0FFF0FFF0FFF0FFF0FFF0FFF0F6D
:10032000FF0FFF0FFF0FFF0FFF0FFF0FFF0FFF0F5D
:10033000FF0FFF0FFF0FFF0FFF0FFF0FFF0FFF0F4D
:10034000FF0FFF0FFF0FFF0FFF0FFF0FFF0FFF0F3D
:10035000FF0FFF0FFF0FFF0FFF0FFF0FFF0FFF0F2D
:10036000FF0FFF0FFF0FFF0FFF0FFF0FFF0FFF0F1D
:10037000FF0FFF0FFF0FFF0FFF0FFF0FFF0FFF0F0D
:10038000FF0FFF0FFF0FFF0FFF0FFF0FFF0FFF0FFD
:10039000FF0FFF0FFF0FFF0FFF0FFF0FFF0FFF0FED
:1003A000FF0FFF0FFF0FFF0FFF0FFF0FFF0FFF0FDD
:1003B000FF0FFF0FFF0FFF0FFF0FFF0FFF0FFF0FCD
:1003C000FF0FFF0FFF0FFF0FFF0FFF0FFF0FFF0FBD
:1003D000FF0FFF0FFF0FFF0FFF0FFF0FFF0FFF0FAD
:1003E000FF0FFF0FFF0FFF0FFF0FFF0FFF0FFF0F9D
:1003F000FF0FFF0FFF0FFF0FFF0FFF0FFF0FFF0F8D
:08040000FF0FFF0FFF0FFF0FBC
:021FFE000500DC
:00000001FF
